:100000000C94A9040C9404260C9404260C94042645
:100010000C9404260C94C6040C94C6040C94C604D8
:100020000C94C6040C94C6040C94AE1D0C94BF250D
:100030000C94C6040C94C6040C94C6040C947E253F
:100040000C94C6040C94C6040C94CC1D0C94C604E9
:100050000C94C6040C94C6040C94C6040C94C604F8
:100060000C94C6040C94C6040C94C6040C94C604E8
:100070000C94C6040C94C6040C94C6040C94C604D8
:100080000C94C6040C94C6040C94C6041A00D2083E
:100090000800CC080700CD0A0900C6080B00340A86
:1000A0000C007B0B1800000A1900C90998008F0882
:1000B00099006C081E015B0B9E004D0B0000B208FE
:1000C0001A04A2090901C6080B067B090C023C0AA6
:1000D0000801CC081801000A1901C90998018F0804
:1000E00099016C081E00D8080001B2080C016E09C5
:1000F0001E03DC0A0002B2081E023C0A0003B2081A
:100100001804000A1904C9091E05550A1A017809BC
:100110000004B2081E0178090005B2081806000A9A
:100120001906C9091E0116090B0175090006B20856
:100130001807000A1907C9091E085B0807015C08AF
:100140000007B2081E075A080001B2088C00C00060
:10015000EC00F800000114011C0130014401B20858
:10016000971070141F1065104A10E60FFE0119FD5C
:10017000010CFB010BF70109EF0118DF0107BF01BB
:10018000087F011AFF001EEF8198FE8199FF809E73
:100190000000004D454D2031004D454D2032004DB1
:1001A000454D2033004D454D2034000000176917A0
:1001B0001775200B69200B692B1169340B75340BF3
:1001C0000000000001004C3D4C054C3D4C024C3DF4
:1001D0004C014C3D05004C4302004C4301004C4394
:1001E0004C054C434C024C434C014C434B054C4397
:1001F0004B024C434B014C4305001D4302001D4381
:1002000001001D43054C1D43024C1D43014C1D4381
:100210004B051D434B021D434B011D430500254368
:100220000200254301002543054C2543024C25438C
:1002300000006A1876216A216A2C6A357635112504
:10024000241125241E1F22231917000060EA30758F
:10025000E02E70178813D007E803F401C80064008B
:10026000320014000A000500409C204E1027A00F09
:10027000D007E8039001C800C800C800C800C80043
:10028000C8000101010101010101010102040A1478
:1002900028646464646464646464C8C8C8C8FFFE95
:1002A000FCF8F0E0C0800103070F1F3F7FFF07024B
:1002B0000207081C3E1C1C1C3E1C080000143E7F4C
:1002C0003E140000000050487F09110000000005A6
:1002D000097F484400000000387C7C7C3800000026
:1002E0000000000000000000000000000000005FAF
:1002F00000000007000700147F147F14242A7F2ABF
:100300001223130864623649552250000503000089
:10031000001C2241000041221C00082A1C2A080857
:10032000083E08080050300000080808080800606F
:1003300060000020100804023E5149453E00427F03
:10034000400042615149462141454B311814127F0A
:100350001027454545393C4A494930017109050393
:100360003649494936064949291E003636000000FB
:1003700056360000000814224114141414144122AB
:100380001408000201510906324979413E7E1111DB
:10039000117E7F494949363E414141227F414122F8
:1003A0001C7F494949417F090901013E41415132C0
:1003B0007F0808087F00417F41002040413F017FC6
:1003C000081422417F404040407F0204027F7F04A6
:1003D00008107F3E4141413E7F090909063E4151D7
:1003E000215E7F09192946464949493101017F01AA
:1003F000013F4040403F1F2040201F7F2018207FAA
:1004000063140814630304780403615149454300ED
:10041000007F4141020408102041417F0000040296
:1004200001020440404040400001020400205454B6
:1004300054787F484444383844444420384444483D
:100440007F3854545418087E090102081454543C4F
:100450007F0804047800447D40002040443D0000B3
:100460007F10284400417F40007C041804787C08F9
:1004700004047838444444387C14141408081414D0
:10048000187C7C080404084854545420043F444019
:10049000203C4040207C1C2040201C3C4030403C04
:1004A00044281028440C5050503C4464544C4400A0
:1004B0000836410000007F000000413608000808AF
:1004C0002A1C08081C2A08083E5149453E00427F64
:1004D000400062514949462141494D331814127F69
:1004E0001027454545393C4A494931017109050301
:1004F0003649494936464949291E0036360000002A
:100500004034000008142241001414141414004153
:1005100022140802015905023E415D594E7C121118
:10052000127C7F494949363E414141227F41414148
:100530003E7F494949417F090909013E41415171C5
:100540007F0808087F00417F4100204040403F7FF6
:10055000081422417F404040407F020C027F7F040C
:1005600008107F3E4141413E7F090909063E415145
:10057000215E7F09192946264949493201017F0137
:10058000013F4040403F1F2040201F7F2018207F18
:100590006314091463030478040361514945437FDC
:1005A0007F41414102040810204141417F7F1008F2
:1005B0000408104040404040000102040020545410
:1005C00054787F4444443838444444443844444490
:1005D0007F3854545458087E090902004C9292FC0A
:1005E0007F0404047800447D40002040443D007FA7
:1005F0001010284400417F40007C0438047C7C04B7
:1006000004047838444444387C141414080814143E
:10061000147C7C080404044854545424043F444487
:10062000203C4040207C1C2040201C7C4030407CF2
:1006300044281028440C5050503C4464544C44000E
:100640000060600000000000000808080808008042
:10065000008000400220021002080224824342C4AB
:1006600032080E100220006000C000400000604010
:100670001F48204840487FFF424842404FF8440806
:100680004A08447F4388450948EA1E4800000000A4
:1006900000000FF804480448044804483FFF444859
:1006A0004448444844484FF84000700000000100AE
:1006B0000100010201020102410281027FE20112F6
:1006C000010A010601020100018001000000000092
:1006D00000503F4F014A0148FFFF214861483F4811
:1006E00000000FFC400080007FFF00000000008041
:1006F00000400020FFF8000700220018000CFFFB5C
:10070000044804480448046806480408000000003F
:1007100000000000FFF844484448444C444B444A1D
:10072000444844484448FFF8000000000000020824
:10073000018800687FFF0028204822102C482144AF
:100740002E4330442848275022102010000000007B
:10075000000007FC0208020802080208FFFF020866
:1007600002080208020807FC000800000000004020
:100770000042004C7FC420001022FFAA0AAA0AAA45
:100780000ABF4AAA8AAA7FAA002200200000080005
:10079000061201920072FFFF00510081FFF2049CDB
:1007A0000490049F449084987FF40002000000406D
:1007B0000020FFF800078212431022F212520A5260
:1007C00007D21A52225E6250C2504210000000004E
:1007D0000000580038000000000000000000000089
:1007E0000000000000000000000000000000000009
:1007F00000000000000000000000000000000000F9
:10080000000000000000000000000000000007F8E9
:100810000FFC1C0E18061C0E0FFC07F8000002004F
:1008200006001FFE1FFE00000000060E0E1E183EF2
:10083000106618C60F86070604080C0C18C618C6E2
:1008400019E60F3C0738007000F003300C301FFE33
:100850001FFE00301F981FCC19861986198618FCB8
:10086000187807F80FFC1986198619860CFC04788D
:10087000180E181E187819C01F001E001C0006381C
:100880000F7C19C6108219C60F7C063807880FCC5A
:1008900018E6186618C60FFC07F8000000060006E8
:1008A0000000000000000000000000000000000048
:1008B0000000000000001FFE1FFE0E00070001FEEA
:1008C00001FE07000E001FFE1FFE1FFE1FFE00C0E0
:1008D00001C003E007F00E381C1C180E10061FFEA6
:1008E0001FFE1FFE00C000C000C000C01FFE1FFE94
:1008F0001FFE0306030E031E0336036603C60386AC
:10090000030600000000FFFEFFFEFFFEC300C30061
:10091000C300C300C300C000C000C000C000E000AE
:10092000F000FFFFFFFFF000E000C000C000066025
:100930000660066006600660066006600660066087
:100940000660008844CC22AA66EE119955DD33BBBF
:1009500077FF11241FBECFEFD0E1DEBFCDBF12E085
:10096000A0E0B1E0EEECFDE402C005900D92A836E7
:10097000B107D9F71DE0A8E6B2E001C01D92A03E84
:10098000B107E1F70E94C8040C94E5260C9400001E
:100990000E9446050E9433050E94CB050E94C205B5
:1009A0000E94C5050E94610580E091E060E00E9420
:1009B000910578940E94AB070E945E1AB99A86E965
:1009C0008093AE05C19A8AEF90E00E945D0DC198B8
:1009D0008AEF90E00E945D0D8091AE05815080937A
:1009E000AE05882379F788EB9BE00E945D0D86E9D0
:1009F0008093AE05C19A8AEF90E00E945D0DC19888
:100A00008AEF90E00E945D0D8091AE058150809349
:100A1000AE05882379F7B9980E9499110E9439127E
:100A20000E94CF101092AE058091AE058823A1F4EC
:100A3000809106028F3098F00E94B5130E9426061E
:100A40008091710290917202892B71F30E94E607E6
:100A50008091AE05882361F30E94451CE5CF0E947A
:100A6000B712ECCF089580E485BF8EE080936D00CF
:100A700087E080936C0088E080BD8AEA80936A00FA
:100A80001ABE8FE089BF8FEF88BF08951BBA1ABACC
:100A900083E088BB81E987BB15BA8FEF84BB8FE009
:100AA00082BB11BA13B888E382B988E080936200F0
:100AB00080EE80936100109265008FE18093640066
:100AC00008951BB888E98AB986E080939500109252
:100AD00090008FE189B9089510929B0088E180937E
:100AE0009A0086E080939D00109298008FE1809399
:100AF000990008955D9BFECF8CB90895982F809141
:100B00009B0085FFFCCF90939C0008955F9BFECFD8
:100B10008CB1089580919B0087FFFCCF80919C0051
:100B20000895FC01662371F090819923B1F08091C2
:100B30009B0085FFFCCF90939C0031969081992378
:100B4000B1F7089580818823E1F35D9BFECF8CB9D6
:100B5000319680818823C9F7089508958BB1881F45
:100B60008827881F089580919B00881F8827881FE9
:100B7000089580919B0087FD02C080E008958091D8
:100B80009C00089580E188B9089584E087B916B87B
:100B900010928E0008958DE183BF12BE8BE981BF54
:100BA0001FBC89E18EBD10927A001DBC1CBC1BBC11
:100BB0001ABC19BC18BC109279001092780017BCAE
:100BC00016BC99E095BD14BC81E083BD89EA809391
:100BD0008B0090938A0010928C00109289001092E2
:100BE00088001092870080E680938600109285002E
:100BF0001092840010928300109282001092810063
:100C00001092800082E087BF10927D008FEF86BF38
:100C10008FE380937C00089508959C01E199FECFB5
:100C20003FBB2EBB6DBBF894E29AE19A789408958D
:100C30009C01E199FECF3FBB2EBBE09A8DB3089596
:100C4000E3ECFFEFE491E093BC05089580916E0220
:100C5000882309F4BCC010926E0280B38F708F306D
:100C6000E1F4809175028150809375028091730246
:100C7000882351F080916F029091700290937202DC
:100C8000809371021092730210926D02109274029E
:100C9000109277021092760208958EE18093750289
:100CA00080EC809362000E9418200E9418200E940D
:100CB00018200E9418200E94182020916F02309165
:100CC000700280B390E08F709070207F3170822B23
:100CD000932B9093700280936F0280916F0290919A
:100CE000700282959295907F9827807F98279093A5
:100CF000700280936F0280EA809362000E94182045
:100D00000E9418200E9418200E9418200E9418207B
:100D100020916F023091700280B390E08F709070DC
:100D2000207F3170822B932B9093700280936F02FF
:100D300080916F029091700282959295907F982792
:100D4000807F98279093700280936F0280E6809353
:100D500062000E9418200E9418200E9418200E9401
:100D600018200E94182020916F023091700280B3E9
:100D700090E08F709070207F3170822B932B909336
:100D8000700280936F02109262008091BB05853CD7
:100D900019F086E08093820220916F0230917002F8
:100DA00080917602909177022817390789F4809113
:100DB0006D028F5F80936D0280916D028330B8F475
:100DC00080916D02823019F481E08093730208955E
:100DD00080916F02909170029093770280937602D7
:100DE00010926D0210927402109273020895809115
:100DF0006D028F3F61F782E080936D0280917402F3
:100E00008F5F8093740280917402843001F7809127
:100E10006F029091700290689093720280937102B9
:100E200083E080937402109273020895882389F5F9
:100E300080916500877F80936500C098442389F185
:100E400080916500826080936500809165008E7F4F
:100E5000809365008091650080618093650065BB2B
:100E600081E090E00E945D0D809165008F7E80930F
:100E70006500809165008E7F80936500809165009C
:100E80008D7F8093650081E090E00E945D0D8FEF83
:100E90000895C09880916500886080936500442320
:100EA00079F680916500816080936500809165008E
:100EB0008D7F80936500CECF1F93982F6623C9F551
:100EC00080916500816080936500809165008D7FD1
:100ED000809365009923C9F18091650088608093B3
:100EE0006500C09A8091650080618093650014BAA6
:100EF00081E090E00E945D0D13B381E090E00E94DC
:100F00005D0D8FEF84BB809165008E7F80936500BF
:100F1000809165008D7F80936500809165008F7E54
:100F20008093650081E090E00E945D0D812F1F910C
:100F300008958091650082608093650080916500CE
:100F40008E7F80936500992339F680916500877FB5
:100F500080936500C6CF809165008B7F809365008C
:100F600088EE93E00E945D0D80916500846080931F
:100F7000650084E690E00E945D0D80E06FE340E054
:100F80000E9416078823C9F380E06FE341E00E94C6
:100F900016078823C9F30895AB01FB01259134910D
:100FA0002115310549F410C04D5F5F4FFA012591BD
:100FB00034912115310541F028173907A9F74E5F03
:100FC0005F4FFA018491089580E008958091710245
:100FD00090917202892B09F443C0409171025091A3
:100FE00072022CE631E0F90185919491009749F461
:100FF0003BC02D5F3F4FF90185919491009709F413
:1010000033C048175907A9F72E5F3F4FF901949154
:101010009093790280917C02E82FF0E0EE0FFF1FA1
:10102000E45BFE4F25913491F9018491882329F4E2
:1010300018C0349684918823A1F09817D1F731967F
:10104000849180937C02CF010196FC01259134911B
:10105000F9010995109279021092720210927102B0
:10106000089522EB38E0F4CF90E0D2CFFB01DA0113
:101070009491992329F40EC034969491992351F0B8
:101080009817D1F7319684918C93319625913491AC
:10109000C901089522EB38E0C901089510927C023D
:1010A0001092790210927A0281E080937B02809301
:1010B0007D02089508950895089590917B02292F47
:1010C00030E0220F331F225A3E4FF90145915491CF
:1010D00090E0FA010995089580918202882339F001
:1010E000809105028823D1F0815080930502809180
:1010F0007C02882339F485E08093780280E00E94A6
:101100005D080895813051F480917B02823031F482
:1011100085E08093780280E00E945D0808958091C8
:101120008202882339F0809105028823D1F0815012
:101130008093050280917C02882339F485E08093B6
:10114000780281E00E945D080895813051F4809119
:101150007B02823031F485E08093780281E00E9446
:101160005D080895089580917D020E94BA188091CB
:101170007B020E94BA1880917B0280937D0289E6EF
:1011800067E147E127E20E948219089584E0809395
:101190007B020E94B308089582E080937B020E9444
:1011A000B308089583E080937B020E94B3080895FA
:1011B0000F931F938091800298E08927809380028B
:1011C00000E010E0C8010E94180680930602C801E2
:1011D00001960E94180680930702C80102960E9499
:1011E000180680930802C80103960E94180680938F
:1011F0000902C80104960E94180680930A02C801D9
:1012000005960E94180680930B02C80106960E945C
:10121000180680930C02C80107960E941806809356
:101220000D020E944B111F910F9108950F931F9370
:10123000CF93DF938091A80590E020E231E0829F78
:101240008001839F100D929F100D11248091B20593
:101250009091B305080F191FC6E0D2E0C8010E94A3
:10126000180689930F5F1F4F42E0CE30D407B1F7C5
:101270000091B2051091B305005E1F4F8091A80543
:1012800090E020E231E0AC01429FC001439F900D0D
:10129000529F900D1124080F191FC0E0DFE0C80114
:1012A0000E94180689930F5F1F4F50E1C030D50789
:1012B000B1F780E09EE09093B7058093B6050E9459
:1012C000C8140E944B110E94780D0E9439120E948E
:1012D000CF10DF91CF911F910F9108950E94C814F4
:1012E0000E944B110E94CF1008950E946E0908952C
:1012F0000E946E0908950E947A1985E06AE04AE02A
:1013000051E00E9462194091A8054F5F40638AE452
:101310006AE00E94061985E06EE146E151E00E9414
:10132000621985E068E248E251E00E94621985E0B6
:1013300062E348E351E00E94621980EC99E00E9468
:10134000EB1908950E947A1985E06AE048E451E0BB
:101350000E9462194091A8054F5F40638DE56AE0E5
:101360000E94061985E06EE146E151E00E94621993
:1013700085E068E247E551E00E94621985E062E39A
:1013800044E651E00E94621980EC99E00E94EB195A
:10139000089580910502882351F080917C0281306C
:1013A00039F0813058F08430D1F0863071F00895F2
:1013B00080917B02823011F08430C9F781E0809304
:1013C000780280E00E945D0808958091A805815010
:1013D0008093A8058F3F81F00E947B09089580913A
:1013E000A80581508093A8058F3F19F485E080936C
:1013F000A8050E94A209089585E08093A805ECCF76
:1014000080910502882351F080917C02813039F06F
:10141000813058F08430C9F0863069F008958091A9
:101420007B02823011F08430C9F781E0809378022A
:101430000E945D0808958091A8058F5F8093A8059C
:10144000863079F00E947B0908958091A8058F5F0E
:101450008093A805863011F41092A8050E94A20975
:1014600008951092A805EECF85E080937B020E943C
:10147000B3080E94000A08950E947A198AE06AE07F
:1014800044E751E00E9462198AE068E241E851E0D5
:101490000E9462198AE062E34EE851E00E946219FC
:1014A00080EC99E00E94EB190895EF92FF920F9360
:1014B0001F93CF93DF930E947A1985E06AE04EE98B
:1014C00051E00E94621980EC99E00E94EB19809132
:1014D000A80590E020E231E0829F8001839F100DFB
:1014E000929F100D11248091B2059091B305080FC1
:1014F000191FC6E0D2E0C80169910E940D060F5F76
:101500001F4F42E0CE30D407B1F70091B6051091DD
:10151000B70500501F4FC091B205D091B305A096FA
:101520008091A80590E020E231E0FC01E29FC0013B
:10153000E39F900DF29F900D1124C80FD91FE12C4D
:1015400021E0F22EEC0EFD1ECE01F80161918F011B
:101550000E940D062196F0E100301F0710F00050A8
:101560001140CE15DF0581F70E947A198AE06AE002
:1015700041EB51E00E9462198AE068E244EC51E0DC
:101580000E94621980EC99E00E94EB19DF91CF91E3
:101590001F910F91FF90EF90089581E080937B025F
:1015A0000E94B308809105028111089580E090E0C7
:1015B00060E80E940D060895EF92FF920F931F932B
:1015C000CF93DF930E947A198AE06AE043ED51E0FD
:1015D0000E94621980EC99E00E94EB1940EC55E002
:1015E000A0ECB9E063E872E0FA0180818C9381811C
:1015F00011968C9311978D010E5F1F4F32E0E32EF1
:10160000F12CE40EF51EEB019A012C593F4F899104
:101610009281892B12968C93129731961196E2172C
:10162000F307A9F7D801AC59BF4F6C597F4FF701A9
:10163000EC59FF4F9A0120583F4F81918D93E2174B
:10164000F307D9F785E0633A780711F0AF01CCCF03
:101650000E94211F182F0E947A191123B9F484E1E6
:101660006AE045EF51E00E9462198AE068E244ECCA
:1016700051E00E94621980EC99E00E94EB19DF9121
:10168000CF911F910F91FF90EF90089584E16AE050
:1016900045EE51E00E946219E8CF8091AE058111BC
:1016A000089581E08093AE050E94780D0E94CF10CE
:1016B0000E94B81C08958091800298E08927809349
:1016C00080020E94150F809182020E947A0580910B
:1016D00005020E947A05089560910C0281E0682756
:1016E00060930C0286E090E00E940D060E94660E58
:1016F0000E94680F089580917B02863031F086E069
:1017000080937B020E94B30808950E946C0B86E0D0
:1017100080937B020E94B3080895861708F4682F0F
:10172000862F0895681708F4682F862F0895FB0107
:10173000982F92959F7090639A3308F0995F9083E9
:101740008F7080638A3308F0895F81831282CF01B2
:101750000895282FFB0164E60E94A326482F80638A
:1017600080838CE99FEF489F402D1124420F842FE6
:101770006AE00E94A326982F90639183282F30E07F
:10178000C901880F991F880F991F880F991F220F71
:10179000331F820F931F481B406342831382CF0184
:1017A0000895EF92FF920F931F93FC017B0160E17C
:1017B00077E20E94AF26D7016C9370E080EF98ED3E
:1017C000689F9001699F300D789F300D11242E0F76
:1017D0003F1FC90168EE73E00E94AF26F7016183E5
:1017E00070E088E19CEF689FF001699FF00D789FA1
:1017F000F00D1124E20FF31FCF0164E670E00E94A8
:10180000AF26D70112966C9370E08CE99FEF689F2A
:101810008001699F100D789F100D11240E0F1F1F5E
:10182000C8016AE070E00E94AF26F7016383862F4B
:1018300090E09C01220F331F220F331F220F331F12
:10184000880F991F280F391F021B130B0483158261
:10185000C7011F910F91FF90EF9008954F925F92F3
:101860006F927F928F929F92AF92BF92CF92DF92B0
:10187000EF92FF920F931F935B016C012A0120E00E
:101880003AEC4AE95BE30E94C326F201208330E090
:1018900040E050E0CA01B90120E036E345E654ECEF
:1018A0000E9484267B018C01EA0CFB1C0C1D1D1D73
:1018B000C801B70120E031EE45EF55E00E94C32694
:1018C000F201218330E040E050E0CA01B90120E09C
:1018D0003FE14AE05AEF0E9484265B016C01AE0CA6
:1018E000BF1CC01ED11EC601B50120E836E948E97B
:1018F00050E00E94C326F201228330E040E050E035
:10190000CA01B90120E839E647E65FEF0E94842664
:101910007B018C01EA0CFB1C0C1D1D1DC801B701CD
:1019200020E432E44FE050E00E94C326F20123831A
:1019300030E040E050E0CA01B90120EC3DEB40EF5F
:101940005FEF0E9484265B016C01AE0CBF1CC01EC1
:10195000D11EC601B50120EA36E841E050E00E9400
:10196000C326F201248330E040E050E0CA01B9010F
:1019700020E639E74EEF5FEF0E9484267B018C0161
:10198000EA0CFB1C0C1D1D1DC801B70120E137E24C
:1019900040E050E00E94C326F201258330E040E0A1
:1019A00050E0CA01B90120EF38ED4FEF5FEF0E9420
:1019B00084265B016C01AE0CBF1CC01ED11EC6018B
:1019C000B50128EE33E040E050E00E94C326F2016A
:1019D000268330E040E050E0CA01B90128E13CEF45
:1019E0004FEF5FEF0E9484263B014C016A0C7B1C89
:1019F0008C1C9D1CC401B30124E630E040E050E0A3
:101A00000E94C326F201278330E040E050E0CA0183
:101A1000B9012CE93FEF4FEF5FEF0E9484267B0175
:101A20008C01E60CF71C081D191DC801B7012AE03E
:101A300030E040E050E00E94C326F201208730E011
:101A400040E050E0CA01B90126EF3FEF4FEF5FEFF2
:101A50000E948426E60EF71E081F191FF201E18678
:101A600012861386C2011F910F91FF90EF90DF90B5
:101A7000CF90BF90AF909F908F907F906F905F902E
:101A80004F900895DF93CF9300D0CDB7DEB79A8300
:101A9000898389819A81892B59F00E942006898146
:101AA0009A8101979A83898389819A81892BA9F7E1
:101AB0000F900F90CF91DF910895DF93CF9300D0D7
:101AC000CDB7DEB79A83898389819A81892B59F0B2
:101AD0000E94182089819A8101979A83898389813C
:101AE0009A81892BA9F70F900F90CF91DF910895DC
:101AF000E3E8F2E0119285E0E33AF807D9F70895B8
:101B0000CF93DF93582F4423B9F1E62FF0E0CF01B4
:101B10008F739070959587959595879595958795F1
:101B200024E630E0829FD001839FB00D929FB00DDC
:101B30001124A50FB11DAD57BD4F6150460F6F5F0A
:101B4000403408F05AC0242F269526952695669590
:101B500066956695261B99F4E770F070E256FD4F86
:101B60008491E42FF0E0E770F070EA55FD4FE491C6
:101B7000E8238C918E2B8C93DF91CF9108952130A7
:101B800009F43DC0E770F070E256FD4F94918C91DE
:101B9000892B8C93ED01CC59DF4F223008F1FE01E7
:101BA000922F92505FEF84E6989F90011124285362
:101BB0003F4F2A0F3B1F5083EC59FF4FE217F307AB
:101BC000D1F7892F90E0019624E630E0BC01629FB6
:101BD000C001639F900D729F900D1124C80FD91FF3
:101BE000E42FF0E0E770F070EA55FD4FE491888152
:101BF0008E2B8883DF91CF9108954FE3A4CFE770B8
:101C0000F070E256FD4F94918C91892B8C93AC59D6
:101C1000BF4FE42FF0E0E770F070EA55FD4FE4911C
:101C20008C918E2B8C93DF91CF91089580910C0233
:101C3000882349F090910D02990F990F109283001B
:101C400090938200089580910B02982F990F980F1E
:101C50009695905E109283009093820008958091F3
:101C60000802982F990F980F9695905E1092850014
:101C70009093840080918202882339F0809105023C
:101C8000882319F081508093050208958091050200
:101C9000882371F080910C02882359F083E087B982
:101CA00088B18C7F88B980910A02882359F0419AC3
:101CB000089584E087B988B18C7F88B980910A0241
:101CC0008823A9F788B1836088B90895E8E3F2E032
:101CD00094913196649180910C02882379F449E3C0
:101CE000892F8F5E0E948D168091AB05882321F08D
:101CF00080910C02813021F0BC9A089545E3F0CF29
:101D0000BC98C49A0895FF920F931F93CF93DF93CB
:101D1000E8E3F2E004913196F490E091090213E0D7
:101D2000E19FF0011124CEE3D2E0EC0FFD1FE4911E
:101D3000802F6F2D4E2F0E948D16E0910902E19F9A
:101D4000F00111243196EC0FFD1FE491802F8B5F81
:101D50006F2D4E2F0E948D1680910902819FC00128
:101D600011240296C80FD91FFE014491802F865F6F
:101D70006F2D0E948D16DF91CF911F910F91FF90D3
:101D800008950F931F93E2E3F2E0149131960491CA
:101D9000E0910602F0E0EE0FFF1FEE0FFF1FE05490
:101DA000FE4FE491812F602F4E2F0E948D16E091FF
:101DB0000602F0E0EE0FFF1FEE0FFF1FEF53FE4F86
:101DC000E491812F8B5F602F4E2F0E948D16E09142
:101DD0000602F0E0EE0FFF1FEE0FFF1FEE53FE4F67
:101DE000E491812F855F602F4E2F0E948D16E09128
:101DF0000602F0E0EE0FFF1FEE0FFF1FED53FE4F48
:101E0000E491812F805F602F4E2F0E948D1680916C
:101E10008202882339F080910502882319F08150CD
:101E2000809305021F910F9108958091800283FD98
:101E30001BC08AE662E04CE40E948D168FE662E0E9
:101E40004CE40E948D1684E762E04CE40E948D16FB
:101E500089E762E04CE40E948D168AE662E044E184
:101E600028E00E94821908958AE662E048E10E9413
:101E70008D168FE662E04FE10E948D1684E762E0E6
:101E80004CE10E948D1689E762E044E10E948D16C4
:101E90008AE662E044E128E00E9482190895809178
:101EA000810265E00E94A326865E6EE344E10E9403
:101EB0007F158091070265E00E94A326865E6EE38F
:101EC00044E10E9460158091070280938102089589
:101ED0001F936EE38091BD05681B81E041E00E9485
:101EE0003C1680910C02882369F510910B026EE379
:101EF000611B81E040E00E943C1687E660E042E022
:101F00002DE30E9482191093BD0580910C02882355
:101F1000A1F480910B02982F990F980F9695905EDF
:101F200010928300909382008091BC05803719F055
:101F300088E0809382021F91089590910D02990F7D
:101F4000990FEECF10910D02D2CF1F931EE3809117
:101F5000B805612F681B80E041E00E943C1680912B
:101F60000802181B80E0612F40E00E943C1690910F
:101F700008029093B805892F880F890F8695805E97
:101F8000109285008093840080918202882339F02A
:101F900080910502882319F08150809305021F91DA
:101FA0000895EAE3F2E094913196649180910A02F7
:101FB000882331F44DEC52E0892F0E948017089558
:101FC00044EC52E0892F0E948017089520910C0262
:101FD000222301F590910B02813001F1609178028A
:101FE000961758F1961B692F222301F560930B0277
:101FF00085E090E00E940D0680918202882339F0EE
:1020000080910502882319F08150809305020E9477
:10201000680F089590910D02813001F76091780268
:10202000690F6F3308F36EE3222301F360930D020F
:1020300087E090E00E940D06DFCF61E0D5CF8130D0
:10204000E1F08091080290917802981790F4891B32
:102050008093080282E090E0609108020E940D06E1
:102060000E94A50F80E060E042E02DE30E9482190B
:10207000089582E080930802EDCF809178029091DC
:102080000802890F809308028F3320F38EE3809338
:102090000802E0CF60910A0281E0682760930A029B
:1020A00084E090E00E940D0680917B020E94BA18A5
:1020B0000E94D10F80917B020E94BA1889E664E3E6
:1020C0004BE029E00E9482190895982F8091050223
:1020D000882311F1913009F1809109028150809398
:1020E0000902882319F483E08093090283E090E0D9
:1020F000609109020E940D0680917B020E94BA182D
:102100000E94830E80917B020E94BA1889E66BE2DE
:1021100047E129E00E9482190895809109028F5FAA
:1021200080930902843010F390930902DFCF81304D
:1021300059F180910602815080930602882301F1B3
:1021400080E090E0609106020E940D0680917B0283
:102150000E94BA180E94C10E80917B020E94BA1898
:1021600087B78F7D87BF8091800283FD02C0109268
:10217000800289E667E147E129E00E94821908951B
:1021800081E080930602DCCF809106028F5F80930E
:1021900006028C31A9F68BE180930602D1CF9F9283
:1021A000AF92BF92CF92DF92EF92FF920F931F9365
:1021B000CF93DF9380E068EB40E00E94160780E059
:1021C00062E440E00E94160780E068EB41E00E9474
:1021D000160780E060E441E00E941607F2ECCF2E83
:1021E000F5E0DF2EE3E8AE2EE2E0BE2E9924760184
:1021F000E50110E06991F70181917F01682B81E091
:1022000040E00E9416071F5F1E33A1F77EE3E72E12
:10221000F12CEA0CFB1CE601EE9686010C591F4FCF
:10222000F70161917F018991682B81E041E00E9473
:102230001607C017D107A1F784E690E0A80EB91ED3
:102240009394192D186B80E0612F40E00E941607CF
:1022500080E0612F41E00E94160780E062E440E0E8
:102260000E94160780E060E441E00E94160798E0B3
:10227000991629F0E0E8F0E0CE0EDF1EB8CFDF912E
:10228000CF911F910F91FF90EF90DF90CF90BF9073
:10229000AF909F9008950F931F93CF93DF930E9469
:1022A000C8140E949F15C6E3D2E0FE0184912196D6
:1022B000FE0164910BEB12E0A8010E9480172397A6
:1022C000FE0184912196FE01649142EB52E00E944E
:1022D00080172796FE0184912196FE016491A80142
:1022E0000E9480178AE16DE343E00E94D0148DE4E0
:1022F0006DE343E00E94D0140E94830E0E94C10E41
:102300000E94D10F0E94660E0E94A50F0E94680FC6
:102310000E944F0F0E94150F80917B020E94BA18F5
:1023200080EC95E00E94EB19DF91CF911F910F9106
:1023300008950F931F931092AB051092BD05109254
:10234000B8051AE501E080E29EE40E94420D039B7D
:1023500002C00093BD05039902C00093B805115057
:1023600091F78091BD05882329F08091B8058823D5
:1023700009F07BC0E3E8F2E0119245E0E33AF407AC
:10238000D9F720E03EE0F90180E881935EE0EF3F7D
:10239000F507D9F73093B5052093B40510927C0268
:1023A0001092790210927A0280E490E09093A40552
:1023B0008093A3058091A3059091A40520E031E0CE
:1023C000A901481B590B5093BF054093BE051092BD
:1023D000A8053093B3052093B20580E090E00E94F9
:1023E00018068093060281E090E00E941806809310
:1023F000070282E090E00E9418068093080283E0C2
:1024000090E00E9418068093090284E090E00E9408
:10241000180680930A0285E090E00E9418068093D7
:102420000B0286E090E00E94180680930C0287E081
:1024300090E00E94180680930D021092800281E0C5
:1024400080937B0280937D02809108028093B8057F
:1024500080910B028093BD058091070280938102D9
:102460000E944B111F910F91089581E08093AB055D
:1024700081CFEF92FF920F931F93CF93DF938091C1
:10248000800283FD0FC08091000E8093000FA1E0B9
:10249000BEE0FD01E050FF4F8D9180838FE0A030C2
:1024A000B807B9F78091800280FD51C08091070282
:1024B0002091B6053091B705280F311D8FE02030EF
:1024C000380719F010F020503140E3E8F2E01192A3
:1024D00085E0E33AF807D9F7E901C050DF4F10E093
:1024E000AEE3EA2E24C00EE3112311F40093AC05F1
:1024F000802F6091AC050E948D0BF82E802F60918B
:10250000AC050E94920B482F0093AC056E2D681B02
:102510004F5F4F19812F0E94800D219680E1C030BE
:10252000D80710F0C0E0DFE01F5F143649F00881E3
:10253000069506950F33B8F60230B0F602E0D4CF18
:10254000DF91CF911F910F91FF90EF9008958091AF
:102550008002886080938002809180028E7F8093C9
:10256000800281E080937C020E94150F9FCF8091B2
:10257000800283FD81C08091800281FF7EC08091B6
:10258000B0059091B105892B09F076C08091AD0519
:10259000E091A905F091AA0580838091A905909109
:1025A000AA0501969093AA058093A90580509F40A3
:1025B00030F080E09EE09093AA058093A905809179
:1025C0000602282F30E0F901EE0FFF1FE65BFD4FFA
:1025D000859194919093B1058093B0058091090203
:1025E0008130A9F08091800282FF72C08091A505A0
:1025F00081508093A5058091A505882309F03CC0F2
:10260000809180028B7F80938002449A089580910C
:10261000AF0581508093AF058091AF05882361F5A8
:102620002E573D4FF90184918093AF052091A90564
:102630003091AA05C90101969093B7058093B6051C
:1026400080509E4030F42F5F3E4F3093B70520936B
:10265000B6058091B6059091B7052FE080309207BE
:1026600039F030F0805091409093B7058093B605D3
:102670000E9439120E94CF100895809180028260DA
:10268000809380028091800284608093800280E841
:102690008093A50580E09EE09093AA058093A9050C
:1026A00080910602E82FF0E0EE0FFF1FE65BFD4F82
:1026B000859194919093B1058093B00581E08093CA
:1026C000AF0587B78F7D87BF0E94460E449A089555
:1026D0008091800285FF32C08091A5058150809352
:1026E000A5058091A505882339F62091A60530918E
:1026F000A7058091A3059091A405281B390B309361
:10270000B7052093B6054EE02030340730F4205052
:102710003F4F3093B7052093B6050E9439120E94AF
:10272000CF101092800280910902833009F0A4CF6B
:10273000809180028160809380020895449B9CCFA9
:102740008091A9059091AA059093A7058093A6056D
:10275000809180028062809380028091A305909195
:10276000A40581958093A50508958091800287FD39
:1027700049C08091800286FF44C08091800284FD20
:1027800035C08091800285FF27C0809180028F7DB7
:10279000809380022091A6053091A7058091A30522
:1027A0009091A405281B390B3093B7052093B605EB
:1027B000FEE020303F0730F420503F4F3093B70504
:1027C0002093B60580910902833061F480918002E4
:1027D00081608093800206C080E09EE09093B70500
:1027E0008093B6050E9439120E94CF1086B782608E
:1027F00086BF87B7826087BF809180028F7B80937E
:10280000800208958091800286FDB3CF809180027E
:1028100083FDAFCF809180028F76809380020E94EB
:10282000460E87B78D7F87BF86B7826086BFE091EF
:102830000602E93109F448C0EA3108F03DC0E73149
:1028400009F44BC0E83109F445C080E09EE0909364
:10285000AA058093A9051092A50580918002846045
:10286000809380028E2F90E0880F991FFC01E55B1A
:10287000FD4FE491E7BD865B9D4FFC01849186BDD1
:1028800086B7806286BF87B7806287BF80918002EB
:1028900086FD09C0809175028823C1F38091800272
:1028A00080618093800287B78F7D87BF809180028F
:1028B0008064809380025DCFEA3149F0EB3109F00A
:1028C000C4CF0E942D20F2CF0E944B24EFCF0E9454
:1028D000F023ECCF0E94B624E9CF0E941D25E6CF5D
:1028E000813009F447C080910702909178029817CF
:1028F000F0F5891B8093070281E090E06091070268
:102900000E940D060E944F0F88E16DE344E323E02F
:102910000E9482198091800283FF28C08091070263
:102920002091B6053091B705280F311D3093B505BC
:102930002093B4058EE02030380730F420503F4F0C
:102940003093B5052093B4058091B4059091B505F9
:102950002FE08030920730F0805091409093B50581
:102960008093B4050E9439120E94CF1008951092EE
:102970000702C2CF8091780290910702890F80935D
:1029800007028C3908F4B8CF8CE980930702B4CFE2
:10299000E0ECF5E0119289E0E03CF807D9F7089502
:1029A000CF93DF934423A1F1E62FF0E0DF01A2955E
:1029B000B295B07FBA27A07FBA27A078B370A80FCE
:1029C000B11DA054BA4F6150460F6F5F403418F5E7
:1029D0008091BB05853C19F085E080938202242F0D
:1029E000269526952695669566956695261BC9F4C7
:1029F000E770F070E256FD4F8491E42FF0E0E7704D
:102A0000F070EA55FD4FE491E8238C918E2B8C9366
:102A1000DF91CF9108954FE38091BB05853CE1F6AE
:102A2000DECF2130B1F1E770F070E256FD4F9491A6
:102A30008C91892B8C93ED01C058DF4F2230E0F050
:102A4000FE0122505FEF30E0C90102969695982F63
:102A50008827979587958A0F9B1F5083E058FF4FD3
:102A6000E817F907D1F72F5F3F4F3695322F22270E
:102A700037952795C20FD31FE42FF0E0E770F07071
:102A8000EA55FD4FE49188818E2B8883DF91CF91A9
:102A90000895E770F070E256FD4F94918C91892B68
:102AA0008C93A058BF4FE42FF0E0E770F070EA5528
:102AB000FD4FE4918C918E2B8C93DF91CF910895F3
:102AC0004423E1F0E62FF0E0E295F295F07FFE2757
:102AD000E07FFE27E078F370E80FF11DE054FA4F35
:102AE000677081E090E0282F01C0220F6A95EAF715
:102AF000622F8081862B81934150D9F7089544231A
:102B0000E9F0E62FF0E0E295F295F07FFE27E07F16
:102B1000FE27E078F370E80FF11DE054FA4F67707C
:102B200081E090E0282F01C0220F6A95EAF7622F1A
:102B300060958081862381934150D9F70895CF9283
:102B4000DF92EF92FF920F931F93CF93DF93A2E454
:102B5000B6E042EC56E022E437E0C2E4D8E062ECB2
:102B600078E08C9184608C931296FA018081806168
:102B700080834E5F5F4FF9018081806480832E5F88
:102B80003F4F8881816088832296FB018081846029
:102B900080836E5F7F4FF6E0A83ABF0711F7CCEC59
:102BA000D5E09CE4E92E96E0F92E8D010C5D1F4FD7
:102BB0006CE477E04CEC57E02CE438E0ACECB8E0A7
:102BC0008CE4C82E89E0D82E8881856588832A9672
:102BD000F7018081856580838AE090E0E80EF91E28
:102BE000F801808185658083065F1F4FFB0180812E
:102BF00085658083665F7F4FFA018081856580836C
:102C0000465F5F4FF901808185658083265F3F4F76
:102C10008C9185658C931A96F601808185618083FD
:102C20008AE090E0C80ED91E96E0C632D90761F658
:102C3000E2ECF5E0808181608193CE17DF07D1F768
:102C4000E2E4F9E080818061819389E0E63AF80767
:102C5000C9F782E060E04DE30E94D01486E660E0B0
:102C60004DE30E94D014DF91CF911F910F91FF90FF
:102C7000EF90DF90CF900895CF93DF93982F882324
:102C8000F9F420E030E0862F869586958695C82F4A
:102C9000D0E0D695DC2FCC27D795C795C20FD31F90
:102CA000C054DA4F442379F0A0E0B0E020E030E0F7
:102CB000462F4770C9F4A8832983DF91CF910895E7
:102CC00027E630E0E0CF992329F52EEA32E0F9013A
:102CD0008491A82FB0E02F5F3F4FF9018491282FF6
:102CE00030E0462F477039F3CD01042E02C0880F23
:102CF000991F0A94E2F702C0220F331F4A95E2F7A8
:102D000088832983FE01E058FF4F90833183DF9150
:102D1000CF91089520EB32E0DACF0F931F93CF933A
:102D2000DF93962F969596959695A92FB0E0B69538
:102D3000BA2FAA27B795A795A80FB11DA054BA4FCF
:102D400085E0489F8001112408531B4F677069F18B
:102D50008FEF90E0982F062E01C0990F0A94EAF7A2
:102D6000792F7095ED01C058DF4F40E050E0F80139
:102D7000E40FF51FE4912E2F30E0062E02C0220F43
:102D8000331F0A94E2F78C918723822B8D938881DD
:102D90008923832B89934F5F5F4F4530510539F766
:102DA000DF91CF911F910F91089520E030E0F8015D
:102DB000E20FF31FE4918C918078E82BED932F5F65
:102DC0003F4F2530310599F7DF91CF911F910F913A
:102DD00008958F929F92BF92CF92DF92EF92FF92CF
:102DE0000F931F93CF93DF93962F96959695969575
:102DF000A92FB0E0B695BA2FAA27B795A795A80F27
:102E0000B11DA054BA4F242F30E0220F331F22955A
:102E10003295307F3227207F3227225B394F47E0BF
:102E2000D42ED62209F452C0E1EEFFEFE491E093F4
:102E3000BB058FEF90E0C82E0D2C01C0CC0C0A947E
:102E4000EAF7BC2CB0948D0100581F4F812C91E003
:102E5000992E8A0E9B1EF90180E2E82EF12CE20EDB
:102E6000F31E31968491319790E04491742F60E085
:102E7000862B972B0D2C02C0880F991F0A94E2F71E
:102E80002C912B21282B2D93E8012881292B299384
:102E90008E0150E0E40188818C210D2C02C0440F8A
:102EA000551F0A94E2F7852B89934E013296EE1551
:102EB000FF05B9F6DF91CF911F910F91FF90EF9031
:102EC000DF90CF90BF909F908F900895E1EEFFEF3D
:102ED000E491E093BB05F90110E2E12EF12CE20E42
:102EE000F31E3196849131978C938491A058BF4FF3
:102EF0008C93AF57B0403296EE15FF0591F7DACFBD
:102F00000F931F93CF93DF938A01962F96959695F3
:102F10009695A92FB0E0B695BA2FAA27B795A79591
:102F2000A80FB11DA054BA4F677069F18FEF90E000
:102F3000982F062E01C0990F0A94EAF7792F709501
:102F4000ED01C058DF4F40E050E0F801E40FF51FFD
:102F5000E4912E2F30E0062E02C0220F331F0A9478
:102F6000E2F78C918723822B8D9388818923832B91
:102F700089934F5F5F4F4930510539F7DF91CF910A
:102F80001F910F91089520E030E0F801E20FF31F48
:102F9000E4918C918078E82BED932F5F3F4F29309F
:102FA000310599F7DF91CF911F910F9108958F927D
:102FB0009F92AF92BF92CF92DF92EF92FF920F93C8
:102FC0001F93CF93DF93362FC42E962F9695969509
:102FD0009695E92EFF24F694FE2CEE24F794E794C0
:102FE000E80EF11C80EC95E0E80EF91E97E0491719
:102FF00009F4B9C084E1289FB00111246A54774FC5
:10300000A7E0DA2ED32209F046C0CC2009F436C05E
:10301000D701FB012491822F8F7090E08E5B964F39
:10302000FC01849122952F70E22FF0E0EE5BF64FC9
:10303000E491807FEF708E2B8C936F5F7F4FFB014D
:103040002491822F8F7090E08E5B964FFC018491CB
:1030500022952F70E22FF0E0EE5BF64FE491A0583E
:10306000BF4F807FEF708E2B8C93AF57B0406F5F58
:103070007F4F8A2F8E198C1508F4CBCFDF91CF911B
:103080001F910F91FF90EF90DF90CF90BF90AF9086
:103090009F908F900895CC2089F38FEF90E0B82E09
:1030A0000D2C01C0BB0C0A94EAF7AB2CA09487014D
:1030B00000581F4F812CF1E09F2E8E0C9F1CD701D2
:1030C000FB012491822F8F7090E08E5B964FFC0164
:1030D000849122952F70E22FF0E0EE5BF64FE491A1
:1030E000807FEF708E2B482F50E06F5F7F4FFB018A
:1030F0008491282F2F7030E02E5B364FF9012491F8
:1031000082958F70E82FF0E0EE5BF64FE491207F20
:10311000EF702E2BF22FE0E04E2B5F2B0D2C02C018
:10312000440F551F0A94E2F78C918A21842B8D93CA
:10313000E8018881852B89938E01822F90E0E4013C
:1031400028812B210D2C02C0880F991F0A94E2F7C9
:10315000292B29934E016F5F7F4F8A2F8E198C1573
:1031600008F4AECF8BCF8EE0289FB0011124625FB0
:10317000774F46CF93E0899FA0011124CA0185555E
:103180009E4FFC013491CA0184559E4FFC0124914D
:1031900043555E4FFA014491442321F1822F8695D5
:1031A00086958695A82FB0E0B695BA2FAA27B79531
:1031B000A795A30FB11DA054BA4F27708FEF91E0D0
:1031C00002C0880F991F2A95E2F7382FFD01E058B9
:1031D000FF4F242F8C9183278D93808189278193A2
:1031E0002150C1F70895982F9F7042E459E09A0149
:1031F000290F311DF901249182958F70480F511DBF
:10320000FA018491207F8F70822B08950F931F9372
:10321000CF93DF93962F969596959695A92FB0E02C
:10322000B695BA2FAA27B795A795A80FB11DA05498
:10323000B64F85E0489F80011124085B1D4F6770E1
:1032400069F18FEF90E0982F062E01C0990F0A9434
:10325000EAF7792F7095ED01C058DF4F40E050E05C
:10326000F801E40FF51FE4912E2F30E0062E02C086
:10327000220F331F0A94E2F78C918723822B8D93C0
:1032800088818923832B89934F5F5F4F4530510598
:1032900039F7DF91CF911F910F91089520E030E031
:1032A000F801E20FF31FE4918C918078E82BED9305
:1032B0002F5F3F4F2530310599F7DF91CF911F9157
:1032C0000F9108950F931F93CF93DF93182F062F1D
:1032D000EA014881442349F0812F602F0E9406199A
:1032E00021961A5F48814423B9F7DF91CF911F914E
:1032F0000F910895E0ECF9E011928DE0E03CF807C1
:10330000D9F708957F928F929F92AF92BF92CF92FA
:10331000DF92EF92FF920F931F93CF93DF93A82E2C
:10332000762E7A94720E769476947694B62EB6941F
:10333000B694B694AA94EA2CE40EA3947B14E8F114
:10334000C62FD0E0C295D295D07FDC27C07FDC2786
:10335000C078D370CA0DD11DC054DA4F50E8852E05
:10336000912C841A910830ECC32E3FEFD32EEA142F
:10337000F0F028EBF22EFB280A2D10E0003408F0C4
:1033800011E080E06F2D412F0E9416071C9D602DDB
:103390001124600F606480E0412F0E94160781E0D5
:1033A0006991412F0E9416070F5FE01630F7B39422
:1033B0007B1418F0C80DD91DDACFDF91CF911F9182
:1033C0000F91FF90EF90DF90CF90BF90AF909F90C4
:1033D0008F907F900895DF92EF92FF920F931F934B
:1033E000CF93DF93182F092F80E060EC40E00E941C
:1033F00016078823C9F380E060EC41E00E941607BD
:103400008823C9F380E068EB40E00E941607882318
:10341000C9F380E060E440E00E9416078823C9F306
:1034200080E068EB41E00E9416078823C9F380E042
:1034300060E441E00E9416078823C9F3812F902F92
:103440009C017901DD24E70110E081E0688140E022
:103450000E9416078823C9F321961F5F1034A9F72D
:10346000E701C05CDF4F870100581F4F81E0688192
:1034700041E00E9416078823C9F32196C017D1079F
:10348000A9F77E01D3941D2D186B80E0612F40E0D9
:103490000E9416078823C9F380E0612F41E00E9453
:1034A00016078823C9F388E0D81669F6DF91CF9113
:1034B0001F910F91FF90EF90DF900895E0ECF5E001
:1034C000119289E0E03CF807D9F71092820280E17E
:1034D00068E040E00E94E91680E268E041E00E9476
:1034E000E91680E368E042E00E94E91680E468E0C3
:1034F00043E00E94E91680E568E044E00E94E91696
:1035000080E668E045E00E94E91683E16CE147E26D
:103510000E948D1689E16CE147E20E948D168FE1D1
:103520006CE147E20E948D16E0ECFFEFE491E0933E
:10353000B90585E26CE14BE40E948D168BE26CE1EB
:103540004AE10E948D1681E36CE149E20E948D16EA
:1035500087E36CE145E10E948D168DE36CE144E266
:103560000E948D1683E46CE145E10E948D1689E48A
:103570006CE143E10E948D168FE46CE148E10E940A
:103580008D16E0EEFFEFE491E093BA0585E56CE17E
:103590004BE40E948D168BE56CE143E10E948D1691
:1035A00081E66CE14FE10E948D1687E66CE14DE10A
:1035B0000E948D16E0EFFFEFE491E093A505E1EFA7
:1035C000FFEFE491E093AD058091A505823429F4E5
:1035D0008091AD058C3409F4A7C08AE065E34EE123
:1035E0000E948D1680E165E34FE30E948D1686E10F
:1035F00065E34CE40E948D168CE165E342E30E9492
:103600008D1682E265E34FE30E948D1688E265E342
:103610004FE30E948D168EE265E344E40E948D160E
:1036200084E365E34CE30E948D168AE365E34FE390
:103630000E948D1680E465E341E30E948D1686E4C6
:1036400065E344E30E948D168CE465E345E30E9444
:103650008D1682E565E342E40E948D1688E565E3F8
:103660004CE40E948D168EE565E346E30E948D16BC
:1036700084E665E34FE30E948D168AE665E345E440
:103680000E948D1680E765E34EE30E948D1686E763
:1036900065E344E30E948D168091B9058F3219F0DD
:1036A00083E0809382028AE06DE246E10E948D16FB
:1036B00080E16DE247E20E948D1686E16DE24AE00C
:1036C0000E948D168CE16DE240E00E948D1682E230
:1036D0006DE246E00E948D1688E26DE242E00E94B3
:1036E0008D168EE26DE240E00E948D1684E36DE25D
:1036F00041E00E948D168AE36DE24BE40E948D1634
:1037000080E46DE240E00E948D1686E46DE249E0BF
:103710000E948D168CE46DE241E00E948D1680ECD3
:1037200095E00E94EB1908958AE065E342E10E946A
:103730008D1680E165E34CE10E948D1686E165E31C
:103740004AE00E948D16E3EFFFEFE491EF708CE109
:1037500065E34E2F0E948D16E4EFFFEFE491EF70CA
:1037600082E265E34E2F0E948D16E5EFFFEFE491B4
:10377000EF7088E265E34E2F0E948D16E6EFFFEFB3
:10378000E491EF708EE265E34E2F0E948D16E7EF15
:10379000FFEFE491EF7084E365E34E2F0E948D16F6
:1037A0008AE365E34BE40E948D16E9EFFFEFE491B5
:1037B000EF7080E465E34E2F0E948D16EAEFFFEF75
:1037C000E491EF7086E465E34E2F0E948D16EBEFD7
:1037D000FFEFE491EF708CE465E34E2F0E948D16AD
:1037E0005BCF8AE068E04AE020910E020E94D71782
:1037F00085E168E04AE020910F020E94D71781E23C
:1038000068E047E0209110020E94D7178CE268E040
:1038100047E0209111020E94D71785E368E047E056
:10382000209112020E94D7178EE368E047E02091B2
:1038300013020E94D71789E468E047E02091140240
:103840000E94D71782E568E047E0209115020E94A8
:10385000D7178BE568E047E0209116020E94D71742
:1038600086E668E04AE0209117020E94D71781E7B8
:1038700068E04AE0209118020E94D7178AE068E0C9
:103880004EE62CE10E948219089580E760E046ED43
:1038900052E00E94801780E760E049E028E00E9443
:1038A00082191092C40D1092C50D1092C60D10927F
:1038B000C70D0E94132680E760E04FED52E00E94A2
:1038C000801780E760E049E028E00E94821960915B
:1038D000C40D7091C50D8091C60D9091C70D4EEC31
:1038E0005DE00E942E0CE1EDFDE0A0E1B2E090E091
:1038F0002BE007C091E0319611968DE0E83DF80786
:1039000069F080818C939923B1F7882399F72C93E0
:10391000319611968DE0E83DF80799F70E94F11B6A
:1039200080EC8093620084E690E00E945D0D8099B7
:103930000EC080916D028F5F80936D0280916D0249
:10394000823059F080E69AEE0E945D0D0895109243
:103950006D0280916D028230A9F71092AE050E942F
:10396000CB050E94C8140E9499111092620008951C
:103970000E94C8140E94F11B85E064E343E70E94A3
:10398000601585E067E348E10E948D168BE067E3F0
:103990004FE10E948D1681E167E34CE10E948D1694
:1039A00087E167E344E10E948D1680E267E34BE222
:1039B0000E948D1686E267E34FE10E948D168CE22D
:1039C00067E34BE10E948D1682E367E34DE20E94BC
:1039D0008D168BE367E34DE00E948D1681E467E36B
:1039E0004EE00E948D168AE467E343E20E948D1642
:1039F00080E567E343E10E948D1686E567E34FE1CA
:103A00000E948D168CE567E340E20E948D1682E6E7
:103A100067E345E10E948D1680EC95E00E94EB196A
:103A20001FBC86E08EBD8CE085BD14BC8CE783BDD9
:103A300010928B0081E080938A0017BE10927D0067
:103A40008FEF86BF8FE380937C00089515BC1BB871
:103A500088E98AB986E080939500109290008FE102
:103A600089B908955D9BFECF8CB90895CF93DF93FC
:103A7000DC01662309F180E090E0C1E2D0E1FC9135
:103A8000E0E09C012E273F2748E003C041509C0105
:103A900051F0C901880F991F37FFF8CF8C279D2758
:103AA00041509C01B1F7615011F01196E8CF9C0193
:103AB000C901DF91CF91089520E030E0F9CF982F30
:103AC000DB015D9BFECF81E08CB95D9BFECF9CB995
:103AD0005D9BFECF90959CB980E0FD01E80FF11D44
:103AE000E0815D9BFECFECB98F5F8038B1F720E0BD
:103AF00030E050E8E1E2F0E17C9160E0C901862726
:103B0000972748E003C0415051F0C9019C01220FA2
:103B1000331F97FFF8CF2E273F274150B1F7515061
:103B200011F01196E9CF5D9BFECF3CB95D9BFECFB6
:103B30002CB908955D9BFECF84E08CB9089515BC27
:103B400010BE82E084BD86B7806C86BF87B7806474
:103B500087BF1092690285E085BD08951F920F927C
:103B60000FB60F9211248F9382E084BD8091690279
:103B70008F5F8093690281508B3940F01092690207
:103B800015BC809168028460809368028F910F90C9
:103B90000FBE0F901F9018951F920F920FB60F92A5
:103BA00011248F93DF93CF930F92CDB7DEB78CB1F3
:103BB0008983809168028068809368028981833458
:103BC00091F08981863049F00F90CF91DF918F91EC
:103BD0000F900FBE0F901F90189580916802826021
:103BE00080936802F1CF80916802816080936802BF
:103BF000EBCF0895EF92FF920F931F93DF93CF9334
:103C00000F92CDB7DEB7182F7B0192E005E015BC0F
:103C100010BE94BD86B7806C86BF87B7806487BFAF
:103C20001092690205BD809168028B7F80936802C3
:103C30008091680287FD14C08091680282FFF8CFEE
:103C400080916802887F809368021092690280E008
:103C50000F90CF91DF911F910F91FF90EF900895FA
:103C6000809168028F77809368028091680281FD5D
:103C700021C08091680280FF13C08091680282FD9C
:103C80000FC0812FB70199830E945F1D10926902B6
:103C900015BC80916802887F809368029981B7CFB4
:103CA0001092690215BC80916802887F8093680237
:103CB00080E0CECF15BC1092690280916802887FA7
:103CC0008093680281E0C4CFCF93DF93FC01209101
:103CD0006A02808190E002C0959587952A95E2F767
:103CE00080FF62C030E8EF01219620916A02818155
:103CF00090E002C0959587952A95E2F780FD3064A3
:103D0000DE01119620916A02898190E002C09595AA
:103D100087952A95E2F780FD3062FD01319620916A
:103D20006A0211968C9190E002C0959587952A952C
:103D3000E2F780FD3061DF01119620916A028181F6
:103D400090E002C0959587952A95E2F780FD38604E
:103D5000FD01319620916A0211968C9190E002C08B
:103D6000959587952A95E2F780FD3460DF011196DD
:103D700020916A02818190E002C0959587952A95ED
:103D8000E2F780FD326020916A0211968C9190E0FA
:103D900002C0959587952A95E2F780FD3160832FC3
:103DA0008095DF91CF91089530E09DCFDF92EF9223
:103DB000FF920F931F93CF93DF93EC017B018A0156
:103DC00041155105A9F177E0D72E06C001501040EA
:103DD00079F10894E11CF11CCE010E94641EF701E8
:103DE0008083289680916B0290916C020896909344
:103DF0006C0280936B0280916B0290916C02803810
:103E0000910521F710926C0210926B0280916A0268
:103E1000815080936A02C058D04080916A028F3FDF
:103E2000A9F6D0926A02C058D0400150104089F6DD
:103E3000CE01DF91CF911F910F91FF90EF90DF9016
:103E40000895CF92DF92EF92FF920F931F93DF932B
:103E5000CF93CDB7DEB7C058D0400FB6F894DEBFD1
:103E60000FBECDBF1092680210926C0210926B02CE
:103E700087E080936A0220E030E08E010F5F1F4FE1
:103E8000F801E20FF31FD901A85DBD4F8C9180832B
:103E90002F5F3F4F2E33310599F780E49DE0BE013F
:103EA000615C7F4F42E450E00E94D61E7C0181E0BD
:103EB000B8010E945F1D81E0B8010E94FA1D8823AD
:103EC00089F480E0C058DF4F0FB6F894DEBF0FBE14
:103ED000CDBFCF91DF911F910F91FF90EF90DF90B9
:103EE000CF900895C701B80140E850E00E94D61E67
:103EF0007C0182E0B8010E945F1D82E0B8010E944F
:103F0000FA1D8823F1F2C701B80140E850E00E9491
:103F1000D61E7C0183E0B8010E945F1D83E0B801DA
:103F20000E94FA1D882369F2C701B80140E850E0F9
:103F30000E94D61E7C0184E0B8010E945F1D84E0CF
:103F4000B8010E94FA1D882309F4BBCFC701B8014C
:103F500040E850E00E94D61E7C0185E0B8010E9436
:103F60005F1D85E0B8010E94FA1D882309F4A9CFDE
:103F7000C701B80140E850E00E94D61E7C0186E0EF
:103F8000B8010E945F1D86E0B8010E94FA1D8823D7
:103F900009F497CFC701B80140E850E00E94D61E4F
:103FA0007C0187E0B8010E945F1D87E0B8010E9494
:103FB000FA1D882309F485CFC701B80140E850E015
:103FC0000E94D61E6C0188E0B8010E945F1D88E047
:103FD000B8010E94FA1D882309F473CFFF24EE2450
:103FE000EA9407C0F801EF0DF11DE082F394F7FCAD
:103FF0000DC08DE38F15B0F3C601B8014EE350E05C
:104000000E94D61E6C018EE3F80EF0CF89E0B80155
:104010000E945F1D89E0B8010E94FA1D882309F4FF
:1040200050CF5D9BFECF84E08CB981E04BCF0895EB
:104030000000000000000000000000000000000080
:104040000000000000000000000000000000000070
:1040500000000000000000000895AF93BF938F930D
:104060009F93CF93DF93EF93FF93809157008F73CC
:104070008093570080915600806C8093560089E1B0
:1040800085BD81E084BDA0E0BEE0B79900C0B79BCC
:1040900000C00000000089B38D93000089B38D93A8
:1040A000000089B38D93000089B38D93000089B31C
:1040B0008D93000089B38D93000089B38D93000028
:1040C00089B38D93000089B38D93000089B38D93DC
:1040D000000089B38D93000089B38D93000089B3EC
:1040E0008D93000089B38D93000089B38D930000F8
:1040F00089B38D93000089B38D93000089B38D93AC
:10410000000089B38D93000089B38D93000089B3BB
:104110008D93000089B38D93000089B38D930000C7
:1041200089B38D93000089B38D93000089B38D937B
:10413000000089B38D93000089B38D93000089B38B
:104140008D93000089B38D93000089B38D93000097
:1041500089B38D93000089B38D93000089B38D934B
:10416000000089B38D93000089B38D93000089B35B
:104170008D93000089B38D93000089B38D93000067
:1041800089B38D93000089B38D93000089B38D931B
:10419000000089B38D93000089B38D93000089B32B
:1041A0008D93000089B38D93000089B38D93000037
:1041B00089B38D93000089B38D93000089B38D93EB
:1041C000000089B38D93000089B38D93000089B3FB
:1041D0008D93000089B38D93000089B38D93000007
:1041E00089B38D93000089B38D93000089B38D93BB
:1041F000000089B38D93000089B38D93000089B3CB
:104200008D93000089B38D93000089B38D930000D6
:1042100089B38D93000089B38D93000089B38D938A
:10422000000089B38D93000089B38D93000089B39A
:104230008D93000089B38D93000089B38D930000A6
:1042400089B38D93000089B38D93000089B38D935A
:10425000000089B38D93000089B38D93000089B36A
:104260008D93000089B38D93000089B38D93000076
:1042700089B38D93000089B38D93000089B38D932A
:10428000000089B38D93000089B38D93000089B33A
:104290008D93000089B38D93000089B38D93000046
:1042A00089B38D93000089B38D93000089B38D93FA
:1042B000000089B38D93000089B38D93000089B30A
:1042C0008D93000089B38D93000089B38D93000016
:1042D00089B38D93000089B38D93000089B38D93CA
:1042E000000089B38D93000089B38D93000089B3DA
:1042F0008D93000089B38D93000089B38D930000E6
:1043000089B38D93000089B38D93000089B38D9399
:10431000000089B38D93000089B38D93000089B3A9
:104320008D93000089B38D93000089B38D930000B5
:1043300089B38D93000089B38D93000089B38D9369
:10434000000089B38D93000089B38D93000089B379
:104350008D93000089B38D93000089B38D93000085
:1043600089B38D93000089B38D93000089B38D9339
:10437000000089B38D93000089B38D93000089B349
:104380008D93000089B38D93000089B38D93000055
:1043900089B38D93000089B38D93000089B38D9309
:1043A000000089B38D93000089B38D93000089B319
:1043B0008D93000089B38D93000089B38D93000025
:1043C00089B38D93000089B38D93000089B38D93D9
:1043D000000089B38D93000089B38D93000089B3E9
:1043E0008D93000089B38D93000089B38D930000F5
:1043F00089B38D93000089B38D93000089B38D93A9
:10440000000089B38D93000089B38D93000089B3B8
:104410008D93000089B38D93000089B38D930000C4
:1044200089B38D93000089B38D93000089B38D9378
:10443000000089B38D93000089B38D93000089B388
:104440008D93000089B38D93000089B38D93000094
:1044500089B38D93000089B38D93000089B38D9348
:10446000000089B38D93000089B38D93000089B358
:104470008D93000089B38D93000089B38D93000064
:1044800089B38D93000089B38D93000089B38D9318
:10449000000089B38D93000089B38D93000089B328
:1044A0008D93000089B38D93000089B38D93000034
:1044B00089B38D93000089B38D93000089B38D93E8
:1044C000000089B38D93000089B38D93000089B3F8
:1044D0008D93000089B38D93000089B38D93000004
:1044E00089B38D93000089B38D93000089B38D93B8
:1044F000000089B38D93000089B38D93000089B3C8
:104500008D93000089B38D93000089B38D930000D3
:1045100089B38D93000089B38D93000089B38D9387
:10452000000089B38D93000089B38D93000089B397
:104530008D93000089B38D93000089B38D930000A3
:1045400089B38D93000089B38D93000089B38D9357
:10455000000089B38D93000089B38D93000089B367
:104560008D93000089B38D93000089B38D93000073
:1045700089B38D93000089B38D93000089B38D9327
:10458000000089B38D93000089B38D93000089B337
:104590008D93000089B38D93000089B38D93000043
:1045A00089B38D93000089B38D93000089B38D93F7
:1045B000000089B38D93000089B38D93000089B307
:1045C0008D93000089B38D93000089B38D93000013
:1045D00089B38D93000089B38D93000089B38D93C7
:1045E000000089B38D93000089B38D93000089B3D7
:1045F0008D93000089B38D93000089B38D930000E3
:1046000089B38D93000089B38D93000089B38D9396
:10461000000089B38D93000089B38D93000089B3A6
:104620008D93000089B38D93000089B38D930000B2
:1046300089B38D93000089B38D93000089B38D9366
:10464000000089B38D93000089B38D93000089B376
:104650008D93000089B38D93000089B38D93000082
:1046600089B38D93000089B38D93000089B38D9336
:10467000000089B38D93000089B38D93000089B346
:104680008D93000089B38D93000089B38D93000052
:1046900089B38D93000089B38D93000089B38D9306
:1046A000000089B38D93000089B38D93000089B316
:1046B0008D93000089B38D93000089B38D93000022
:1046C00089B38D93000089B38D93000089B38D93D6
:1046D000000089B38D93000089B38D93000089B3E6
:1046E0008D93000089B38D93000089B38D930000F2
:1046F00089B38D93000089B38D93000089B38D93A6
:10470000000089B38D93000089B38D93000089B3B5
:104710008D93000089B38D93000089B38D930000C1
:1047200089B38D93000089B38D93000089B38D9375
:10473000000089B38D93000089B38D93000089B385
:104740008D93000089B38D93000089B38D93000091
:1047500089B38D93000089B38D93000089B38D9345
:10476000000089B38D93000089B38D93000089B355
:104770008D93000089B38D93000089B38D93000061
:1047800089B38D93000089B38D93000089B38D9315
:10479000000089B38D93000089B38D93000089B325
:1047A0008D93000089B38D93000089B38D93000031
:1047B00089B38D93000089B38D93000089B38D93E5
:1047C0008091800280648093800289E085BDFF91A2
:1047D000EF91DF91CF919F918F91BF91AF9108950C
:1047E000AF93BF938F939F93CF93DF93EF93FF93F9
:1047F000C8B7C068D8B7DF77FFEFE2EC84918833A1
:1048000019F081E0809382029091BE05A0E0BEE0A5
:10481000C8BB89B38C93D8BB00000000A395C1F737
:10482000449AC8BB89B38C93A395D8BB449913C051
:10483000C1F780910902813001F18091800284FDED
:104840001CC080917502882B61F380918002806189
:104850008093800212C0EA2FC8BB89B38C93D8BB67
:10486000A39500009A95C1F7E093A605B093A7051C
:1048700080918002806280938002809180028064B7
:1048800080938002FF91EF91DF91CF919F918F9163
:10489000BF91AF910895AF93BF938F939F93EF9381
:1048A000FF939091BE05A0E0BEE0C79A0000000013
:1048B0000000000089B38C93C7980000000000003E
:1048C000000000000000A39581F7449AC79A0000F9
:1048D00000000000000089B38C93A395C7980000E6
:1048E000000000000000449913C081F78091090284
:1048F000813041F18091800284FD24C08091750255
:10490000882B21F3809180028061809380021AC0FD
:10491000EA2FC79A000000000000000089B38C93C2
:10492000C79800000000000000000000A3959A95C1
:1049300081F7E093A605B093A7058091800280627D
:104940008093800280918002806480938002E3EEF5
:10495000FFEF94919A3919F092E090938202FF91BF
:10496000EF919F918F91BF91AF910895AF93BF93B6
:104970008F939F93EF93FF939091BE05A0E0BEE0CD
:10498000C79A43D089B38C93C7983FD00000A395B2
:10499000B9F7449AC79A39D089B38C93A395C7982D
:1049A00045D0449913C0B1F780910902813009F1D3
:1049B0008091800284FD1DC080917502882B51F387
:1049C0008091800280618093800213C0EA2FC79A91
:1049D0001CD089B38C93C79821D0A3959A95B9F729
:1049E000E093A605B093A705809180028062809332
:1049F000800280918002806480938002FF91EF9119
:104A00009F918F91BF91AF91089500000000000029
:104A100000000000000000000000089500000000F9
:104A200000000000000000000000089500000000E9
:104A300000000000000000000895AF93BF938F9323
:104A40009F93EF93FF939091BE05A0E0BEE0C798BF
:104A5000DCDFDBDFDADF89B38C93C79AD6DFD5DF03
:104A6000D4DFA395A1F7449AC798CFDFCEDFCDDF7F
:104A700089B38C93A395C79AC8DFC7DFD7DF449962
:104A800013C091F780910902813029F18091800251
:104A900084FD21C080917502882B31F380918002C2
:104AA00080618093800217C0EA2FC798AEDFADDF28
:104AB000ACDF89B38C93C79AA8DFA7DFAFDFA395DC
:104AC0009A9599F7E093A605B093A7058091800287
:104AD0008062809380028091BA05813119F084E070
:104AE0008093820280918002806480938002FF9193
:104AF000EF919F918F91BF91AF9108950F938F93F5
:104B00009F93AF93BF930FB790910502992B49F1F3
:104B1000809106028F3090F48091B0059091B1059C
:104B2000DC01AB2B29F001978093B0059093B10580
:104B3000C79889B38093AD05C79A13C08091660268
:104B40008A9569F4809167028A9531F48091800298
:104B500080688093800282E08093670282E3809382
:104B6000660280917502882B19F081E080936E02B5
:104B70000FBFBF91AF919F918F910F9118950F9398
:104B8000AF93BF938F939F930FB7C79889B3A091AB
:104B9000A905B091AA058C93A395A093A905B093FC
:104BA000AA05C79A8091A5058A958093A50590913D
:104BB000800292FF06C0A9F49B7F90938002449AE2
:104BC00010C095FD0AC0449913C059F480910902A0
:104BD000813021F094FF05C001C019F490649093D6
:104BE00080020FBF9F918F91BF91AF910F91189548
:104BF000A093A605B093A705906290938002809140
:104C0000BE058093A505EDCF0F930FB78F938091CD
:104C100080028061809380028EE1809375028F9183
:104C20000FBF0F9118958F939F9382E08093DB0DB8
:104C300081E78093DA0D80E084BD80E886BF882715
:104C40008DBD8CBD84E086BF86B782FD1AC086B755
:104C500087FD1FC080917C0085FD29C080917C006C
:104C600082FFF2CF84E080937C008091CC0D83950D
:104C70008093CC0D49F78091CD0D83958093CD0D18
:104C8000E3CF84E086BF8091C60D83958093C60DE7
:104C9000DECF80E886BF8091DA0D9091DB0D019721
:104CA0008093DA0D9093DB0D892BA1F624C080E26E
:104CB00080937C008091C80D8093C00D8091C90DB8
:104CC0008093C10D8091CA0D8093C20D8091CB0D50
:104CD0008093C30D809180008093C80D80918100E6
:104CE0008093C90D8091CC0D8093CA0D8091CD0D1C
:104CF0008093CB0DB3CF8CB58093C40D8DB58093CD
:104D0000C50D9F918F910895629FD001739FF0010F
:104D1000829FE00DF11D649FE00DF11D929FF00D4B
:104D2000839FF00D749FF00D659FF00D9927729F82
:104D3000B00DE11DF91F639FB00DE11DF91FBD010D
:104D4000CF0111240895991B79E004C0991F96178B
:104D500008F0961B881F7A95C9F780950895AA1BBD
:104D6000BB1B51E107C0AA1FBB1FA617B70710F056
:104D7000A61BB70B881F991F5A95A9F78095909588
:104D8000BC01CD010895A1E21A2EAA1BBB1BFD0197
:104D90000DC0AA1FBB1FEE1FFF1FA217B307E4071A
:104DA000F50720F0A21BB30BE40BF50B661F771F72
:104DB000881F991F1A9469F7609570958095909552
:0E4DC0009B01AC01BD01CF010895F894FFCF17
:104DCE000D0A434F4D30204F4B00446973706C6198
:104DDE007920427566005B2B5D5B2D5D202D3E209C
:104DEE0053656C20627566005B4F4B5D202D3E2037
:104DFE00446973706C6179005B534C4F50455D2074
:104E0E002D3E204578697400536176652057462003
:104E1E00746F20427566005B4F4B5D202D3E205314
:104E2E00617665005B562E504F535D202D3E20451A
:104E3E007869740053656E642073637265656E3FA6
:104E4E00005B4F4B5D202D3E2053656E64005B4C26
:104E5E004556454C5D202D3E2045786974005361C2
:104E6E0076696E672077617665666F726D2E2E2E6F
:104E7E0000536176652077617665666F726D20648A
:104E8E006F6E65005B4F4B5D20746F20726574759D
:104E9E00726E0053656E64696E672073637265652A
:104EAE006E2E2E2E0053656E6420737563636573CC
:104EBE007366756C0053656E64206661696C65641B
:104ECE002020200001C8104E2D01001E00200406D7
:104EDE00000102030405060203240D00010203046F
:104EEE000506074B08094523424D3E04000000000D
:104EFE0000003E000000280000008000000040007E
:104F0E00000001000100000000000004000000008D
:104F1E000000000000000000000000000000000083
:084F2E000000FFFFFF00FA0480
:00000001FF
